:1000000019C033C032C031C030C02FC02EC02DC087
:100010002CC02BC02AC029C028C027C026C025C09C
:1000200024C023C022C021C020C01FC01EC01DC0CC
:100030001CC01BC011241FBECFEFCDBFDFE3DEBF4E
:100040001FE3A0E8BFE3E6EBF2E002C005900D92EB
:10005000A238B107D9F72FE3A2E8BFE301C01D9290
:10006000A938B207E1F795D00FC1CACF81B1817F1E
:1000700081B90895CF93DF93811549F01092843FA1
:100080001092853F8CE08093803F1092833FC09117
:10009000843FD091853F2196C093843FD093853F84
:1000A000E091803FE53170F4F0E0EA5BFE4F0994A7
:1000B000DDDF699738F01092843F1092853F82E02F
:1000C0008093803FDF91CF91089581B18A6081B99B
:1000D0002597C0F31092843F1092853F85E0F0CFC2
:1000E000C5DF2A9778F31092843F1092853F87E00E
:1000F000E7CF81B18A6081B9259720F31092843FC0
:100100001092853F8AE0DCCFB1DF6997D8F2109278
:10011000843F1092853F8CE0D3CF0A9A259790F2C6
:100120001092843F1092853F8EE0CACF9FDF2A97BE
:1001300048F21092843F1092853F80E1C1CF0A9A25
:10014000259708F4BFCF1092843F1092853F82E13B
:10015000B7CF8CDF699708F4B5CF1092843F109227
:10016000853F8091833F8F5F8093833F833070F022
:100170001092833F84E1A4CF81B18E6081B96997E9
:1001800008F4A0CF1092843F1092853F1092803FD8
:1001900099CF8EEC80B9009888E08093100466DFD8
:1001A00081B1806C81B9D091813FC1E082B1817011
:1001B000282F2C27811150C0C093823F8091873F08
:1001C0009091883F8F3F980729F001968093873F51
:1001D0009093883F8091863F811561F08091873FA1
:1001E0009091883F8436910528F08091813F8C273B
:1001F0008093813F2093863F8091823F811599F1C2
:1002000081B18E6081B98091813F8D1771F1D0915C
:10021000813F2CDF8FE996E821E08150904020401B
:10022000E1F700C0000081B18E6081B93FE986E846
:1002300091E0315080409040E1F700C0000016DFAF
:100240002FE332E48FE0215030408040E1F700C0DE
:10025000000081E00FDF11C01092823F1092873FB3
:100260001092883FB7CF02DFCECF8091813F8115BA
:1002700021F08091823F811569F383ED90E301972E
:10028000F1F700C0000092CFF894FFCF11CF1ACF42
:100290001CCF18CF17CF24CF15CF2BCF13CF12CF12
:1002A00033CF10CF3ACF0ECF41CF0CCF48CF0ACFAC
:0602B00050CF08CF61CF22
:0202B600020143
:00000001FF
